S123A1007EA13500000000447374416464723A2004507265737320656E74657220616E6445
S123A12020737461727420746170650453746F70206174200486F09702CEA107BDC009BD78
S123A140C01EFFA105BDC021CEA111BDC009BD7FEB810D27037EA1CEBDC021FEA1057FA1A6
S123A160037FA104BD7FE54D27037EA1CEBDA1DA4D27EBBBA10344B7A1037CA10426EEB6AF
S123A180A10316545410B7A103BDA1DA4D27CFB1A10322F56F00BDA1DAB1A103221D86083E
S123A1A0B7A104BDA1DA4D2712B0A103A60046A7007AA10426ED63000820D909FFA105CE88
S123A1C0A12CBDC009CEA105BDC015BDC021BD7FE54D2703BD7FEB7EC0004FF680602B1126
S115A1E04C270EF680602AF84F4C2705F680602BF839F7
S9030000FC
